:020000040800F2
:1000000000060020A1020008B10F0008690F0008D7
:10001000910F0008690F0008890F0008A30200086B
:10002000A3020008A3020008A3020008FD220008A2
:10003000A3020008A3020008A3020008A30200080C
:10004000A3020008A3020008A3020008A3020008FC
:10005000A3020008A30200088D370008B937000882
:10006000E5370008113800083D380008A3020008F1
:10007000A3020008A3020008A3020008A3020008CC
:10008000A3020008A3020008A3020008A3020008BC
:10009000A3020008A3020008A302000869380008B0
:1000A000A3020008A3020008A3020008A30200089C
:1000B000A3020008A3020008A3020008A30200088C
:1000C000A3020008A3020008A3020008A30200087C
:1000D000A3020008A3020008A3020008A30200086C
:1000E000CD380008A3020008A3020008A3020008FC
:1000F000A3020008A3020008A3020008A30200084C
:10010000A3020008A302000841390008A302000866
:10011000A3020008A3020008A3020008A30200082B
:10012000A3020008A3020008A3020008A30200081B
:10013000A3020008A3020008A3020008A30200080B
:10014000A3020008A3020008A3020008A3020008FB
:10015000A3020008A3020008A3020008A3020008EB
:10016000A3020008A3020008A3020008A3020008DB
:10017000A3020008692E0008A3020008A3020008D9
:10018000A3020008A3020008A3020008A3020008BB
:10019000A3020008A3020008A3020008A3020008AB
:1001A000A3020008A3020008A3020008A30200089B
:1001B000A3020008A3020008A3020008A30200088B
:1001C000A3020008A3020008A3020008A30200087B
:1001D000A3020008552E0008A3020008A30200088D
:1001E000A3020008A3020008A3020008A30200085B
:1001F000A3020008A3020008A3020008A30200084B
:10020000A3020008A3020008A3020008A30200083A
:10021000A3020008A3020008A3020008A30200082A
:10022000A3020008A3020008A3020008A30200081A
:10023000A3020008A3020008A3020008A30200080A
:10024000A3020008A3020008A3020008A3020008FA
:10025000A3020008A3020008A3020008A3020008EA
:10026000A3020008A3020008A3020008A3020008DA
:10027000A3020008A3020008A3020008A3020008CA
:10028000A3020008A3020008A3020008A3020008BA
:10029000A3020008A3020008A3020008A3020008AA
:1002A00002E000F000F8FEE772B63A4880F30888F2
:1002B000394880F3098839484EF60851CEF20001DA
:1002C000086040F20000CCF200004EF63471CEF22D
:1002D00000010860BFF34F8FBFF36F8F40F2000043
:1002E000C0F2F0004EF68851CEF200010860BFF374
:1002F0004F8FBFF36F8F4FF00000E1EE100A4EF604
:100300003C71CEF200010860062080F31488BFF330
:100310006F8F02F0B1F802F053F802F0EDFF4FF0EA
:1003200055301F491B4A91423CBF41F8040BFAE784
:100330001C49194A91423CBF41F8040BFAE71A499B
:100340001A4A1B4B9A423EBF51F8040B42F8040B69
:10035000F8E700201749184A91423CBF41F8040BC6
:10036000FAE702F06BF803F04BF8144C144DAC4272
:1003700003DA54F8041B8847F9E700F041F8114C00
:10038000114DAC4203DA54F8041B8847F9E702F038
:1003900053B80000000600200022002000000008E2
:1003A0000000002000060020183D00080022002068
:1003B0005C220020602200207C420020A002000875
:1003C000A0020008A0020008A00200082DE9F04FDA
:1003D0002DED108AC1F80CD0D0F80CD0BDEC108AED
:1003E000BDE8F08F002383F311882846A047002042
:1003F00001F06AFBFEE701F0E5FA00DFFEE700002E
:1004000038B501F03BFF054601F06EFF0446D0B958
:100410000F4B9D4219D001339D4241F2883512BFE6
:10042000044600250124002001F032FF0CB100F049
:1004300077F800F06DFD00F013FC284600F01EF97F
:1004400000F06EF8F9E70025EDE70546EBE700BFA1
:10045000010007B008B500F0D5FBA0F12003584219
:10046000584108BD07B541F21203022101A8ADF8B9
:10047000043000F0E5FB03B05DF804FB38B5202341
:1004800083F311881748C3680BB101F0A3FB002365
:10049000154A4FF47A71134801F060FB002383F38F
:1004A0001188124C236813B12368013B23606368F1
:1004B00013B16368013B63600D4D2B7833B96368FA
:1004C0007BB9022000F096FC322363602B78032B6B
:1004D00007D163682BB9022000F08CFC4FF47A73CB
:1004E000636038BD602200207D0400087C2300206A
:1004F00074220020084B187003280CD8DFE800F0A5
:1005000008050208022000F067BC022000F054BC7D
:10051000024B00225A607047742200207C23002086
:10052000F8B5504B504A1C461968013100F09980CB
:1005300004339342F8D162684C4B9A4240F2918066
:100540004B4B9B6803F1006303F500339A4280F044
:100550008880002000F09EFB0220FFF7CBFF454B78
:100560000021D3F8E820C3F8E810D3F81021C3F82D
:100570001011D3F81021D3F8EC20C3F8EC10D3F805
:100580001421C3F81411D3F81421D3F8F020C3F8C0
:10059000F010D3F81821C3F81811D3F81821D3F8A4
:1005A000802042F00062C3F88020D3F8802022F03F
:1005B0000062C3F88020D3F88020D3F8802042F076
:1005C0000072C3F88020D3F8802022F00072C3F8B4
:1005D0008020D3F8803072B64FF0E023C3F8084D86
:1005E000D4E90004BFF34F8FBFF36F8F224AC2F8E4
:1005F0008410BFF34F8F536923F480335361BFF3EB
:100600004F8FD2F8803043F6E076C3F3C905C3F3C9
:100610004E335B0103EA060C29464CEA8177013927
:10062000C2F87472F9D2203B13F1200FF2D1BFF35C
:100630004F8FBFF36F8FBFF34F8FBFF36F8F536930
:1006400023F4003353610023C2F85032BFF34F8FBD
:10065000BFF36F8F202383F31188854680F30888CA
:100660002047F8BD0000020820000208FFFF010833
:10067000002200200044025800ED00E02DE9F04F78
:1006800093B0B44B2022FF2100900AA89D6800F08F
:10069000E9FBB14A1378A3B90121B0481170C360D6
:1006A000202383F31188C3680BB101F093FA002370
:1006B000AB4A4FF47A71A94801F050FA002383F352
:1006C0001188009B13B1A74B009A1A60A64A1378B1
:1006D000032B03D000231370A24A53604FF0000A8B
:1006E000009CD3465646D146012000F075FB24B14C
:1006F0009C4B1B68002B00F02682002000F082FA41
:100700000390039B002BF2DB012000F055FB039BC1
:10071000213B1F2BE8D801A252F823F09D070008C7
:10072000C507000859080008E9060008E90600089E
:10073000E9060008EB080008BB0A0008D509000814
:10074000370A00085F0A0008850A0008E906000861
:10075000970A0008E9060008090B00083D08000890
:10076000E90600084D0B0008A90700083D0800082D
:10077000E9060008370A0008E9060008E90600084B
:10078000E9060008E9060008E9060008E90600088D
:10079000E9060008E9060008590800080220FFF7EA
:1007A00059FE002840F0F981009B022105A8BAF10A
:1007B000000F08BF1C4641F21233ADF8143000F0B0
:1007C0003FFA91E74FF47A7000F01CFA071EEBDB5A
:1007D0000220FFF73FFE0028E6D0013F052F00F280
:1007E000DE81DFE807F0030A0D101336052304212C
:1007F00005A8059300F024FA17E004215548F9E70D
:1008000004215A48F6E704215948F3E74FF01C0841
:10081000404608F1040800F03FFA0421059005A8BD
:1008200000F00EFAB8F12C0FF2D101204FF00009C0
:1008300000FA07F747EA0B0B5FFA8BFB00F05EFB51
:1008400026B10BF00B030B2B08BF0024FFF70AFEA9
:100850004AE704214748CDE7002EA5D00BF00B0353
:100860000B2BA1D10220FFF7F5FD074600289BD0F6
:100870000120002600F00EFA0220FFF73BFE5FFA8F
:1008800086F8404600F016FA0446B0B10399404697
:100890000136A1F140025142514100F01BFA0028FB
:1008A000EDD1BA46044641F21213022105A83E4694
:1008B000ADF8143000F0C4F916E725460120FFF723
:1008C00019FE244B9B68AB4207D9284600F0E4F997
:1008D000013040F067810435F3E70025224BBA462A
:1008E0003E461D701F4B5D60A8E7002E3FF45CAFD5
:1008F0000BF00B030B2B7FF457AF0220FFF7FAFD31
:10090000322000F07FF9B0F10008FFF64DAF18F08B
:1009100003077FF449AF0F4A08EB0503926893423F
:100920003FF642AFB8F5807F3FF73EAF124BB84578
:10093000019323DD4FF47A7000F064F90390039A79
:10094000002AFFF631AF039A0137019B03F8012B10
:10095000EDE700BF00220020782300206022002065
:100960007D0400087C230020742200200422002043
:10097000082200200C22002078220020C820FFF747
:1009800069FD074600283FF40FAF1F2D11D8C5F1B0
:1009900020020AAB25F0030084494245184428BFD1
:1009A0004246019200F038FA019AFF217F4800F098
:1009B00059FA4FEAA803C8F387027C4928460193F5
:1009C00000F058FA064600283FF46DAF019B05EB96
:1009D000830533E70220FFF73DFD00283FF4E4AE36
:1009E00000F096F900283FF4DFAE0027B846704BC0
:1009F0009B68BB4218D91F2F11D80A9B01330ED018
:100A000027F0030312AA134453F8203C05934046F1
:100A1000042205A9043700F0CDFA8046E7E73846FE
:100A200000F03AF90590F2E7CDF81480042105A80A
:100A300000F006F902E70023642104A8049300F003
:100A4000F5F800287FF4B0AE0220FFF703FD002880
:100A50003FF4AAAE049800F051F90590E6E70023B0
:100A6000642104A8049300F0E1F800287FF49CAE10
:100A70000220FFF7EFFC00283FF496AE049800F048
:100A80003FF9EAE70220FFF7E5FC00283FF48CAECF
:100A900000F04EF9E1E70220FFF7DCFC00283FF40C
:100AA00083AE05A9142000F049F9074604210490FB
:100AB00004A800F0C5F83946B9E7322000F0A2F8E2
:100AC000071EFFF671AEBB077FF46EAE384A07EB28
:100AD0000903926893423FF667AE0220FFF7BAFC23
:100AE00000283FF461AE27F003074F44B9453FF4B7
:100AF000A5AE484609F1040900F0CEF8042105909E
:100B000005A800F09DF8F1E74FF47A70FFF7A2FC1A
:100B100000283FF449AE00F0FBF8002844D00A9BBF
:100B200001330BD008220AA9002000F0A3F9002805
:100B30003AD02022FF210AA800F094F9FFF792FC96
:100B40001C4800F0C7FF13B0BDE8F08F002E3FF443
:100B50002BAE0BF00B030B2B7FF426AE002364218E
:100B600005A8059300F062F8074600287FF41CAE44
:100B70000220FFF76FFC804600283FF415AEFFF718
:100B800071FC41F2883000F0A5FF059800F0EAF909
:100B900046463C4600F0B2F9A6E506464EE64FF062
:100BA000000901E6BA467EE637467CE67822002058
:100BB00000220020A08601000F4B70B51B780C4668
:100BC0000133DBB2012B11D80C4D4FF47A73296835
:100BD000A2FB033222460E6A01462846B0478442F1
:100BE00004D1074B002201201A7070BD4FF4FA7037
:100BF00000F070FF0020F8E7102200207025002090
:100C0000B0230020002307B5024601210DF10700A3
:100C10008DF80730FFF7D0FF20B19DF8070003B033
:100C20005DF804FB4FF0FF30F9E700000A460421AD
:100C300008B5FFF7C1FF80F00100C0B2404208BD17
:100C400030B4054C0A46014623682046DD69034B53
:100C5000AC4630BC604700BF70250020A086010074
:100C600070B50A4E00240A4D01F0E0F93080286882
:100C70003388834208D901F0D5F92B680444013345
:100C8000B4F5003F2B60F2D370BD00BFB22300204B
:100C90008423002001F0A8BA00F1006000F50030C4
:100CA0000068704700F10060920000F5003001F02C
:100CB0001FBA0000054B1A68054B1B889B1A83421C
:100CC00002D9104401F0AEB90020704784230020FF
:100CD000B223002038B50446074D29B128682044C6
:100CE000BDE8384001F0B6B92868204401F0A0F909
:100CF0000028F3D038BD00BF8423002000207047B7
:100D000000F1FF5000F58F10D0F800087047000088
:100D1000064991F8243033B100230822086A81F88B
:100D20002430FFF7BFBF0120704700BF8823002099
:100D3000014B1868704700BF0010005C1B4B024657
:100D4000F0B518681A4BC0F30B06000C1F885C68DE
:100D5000BE4293F9085003D09F89BE4203D10C33A1
:100D60005C6893F908500426124B1F8804338742AD
:100D700008BF13F9025C013EF7D1013A013C0B4672
:100D80000A44934207D214F9016F581C2EB103464E
:100D900000F8016CF5E7184605E02C2482421C702F
:100DA00001D9981C5D70401AF0BD00BF0010005CB6
:100DB00014220020283A0008022804D1054B4FF4E1
:100DC00080129A6170470128FCD1024B4FF4003227
:100DD000F7E700BF00040258022803D1044B102299
:100DE0009A6170470128FCD1014B0222F8E700BF4D
:100DF00000040258022805D1064A536983F0100303
:100E0000536170470128FCD1024A536983F0020301
:100E1000F6E700BF00040258002310B5934203D048
:100E2000CC5CC4540133F9E710BD0000013810B5A3
:100E300010F9013F3BB191F900409C4203D11AB136
:100E40000131013AF4E71AB191F90020981A10BD66
:100E50001046FCE703460246D01A12F9011B00298E
:100E6000FAD1704702440346934202D003F8011BB3
:100E7000FAE770472DE9F8431F4D144607468846A8
:100E800095F8242052BBDFF870909CB395F824307D
:100E90002BB92022FF2148462F62FFF7E3FF95F888
:100EA00024004146C0F1080205EB8000A24228BFA1
:100EB0002246D6B29200FFF7AFFF95F82430A41B6C
:100EC00017441E449044E4B2F6B2082E85F824601C
:100ED000DBD1FFF71DFF0028D7D108E02B6A03EB19
:100EE00082038342CFD0FFF713FF0028CBD100202D
:100EF000BDE8F8830120FBE788230020024B1A7825
:100F0000024B1A70704700BFB0230020102200204F
:100F100010B5104C104800F0DFF821460E4800F0E4
:100F200007F924680D48D4F89020D2F8043843F02B
:100F30000203C2F8043800F0CDFD0949204600F054
:100F400005FAD4F89020D2F8043823F00203C2F84E
:100F5000043810BDF43A00087025002040420F000C
:100F6000FC3A00087047000000B59BB0EFF3098120
:100F700068226846FFF750FFEFF30583014B9B6B38
:100F8000FEE700BF00ED00E008B5FFF7EDFF000051
:100F900000B59BB0EFF3098168226846FFF73CFF7C
:100FA000EFF30583014B5B6BFEE700BF00ED00E054
:100FB000FEE7000030B50A44084D91420DD011F80B
:100FC000013B5840082340F30004013B2C4013F040
:100FD000FF0384EA5000F6D1EFE730BD2083B8ED7F
:100FE000026843681143016003B11847704700006D
:100FF00013B5406B00F58054D4F8A4381A68117802
:10100000042914D1017C022911D1197901231289F3
:101010008B4013420BD101A94C3002F06DF8D4F88B
:10102000A4480246019B2179206800F0DFF902B054
:1010300010BD0000143001F0EFBF00004FF0FF338F
:10104000143001F0E9BF00004C3002F0C1B80000DC
:101050004FF0FF334C3002F0BBB80000143001F009
:10106000BDBF00004FF0FF31143001F0B7BF0000EA
:101070004C3002F08DB800004FF0FF324C3002F0DF
:1010800087B800000020704710B500F58054D4F8F0
:10109000A4381A681178042917D1017C022914D1C7
:1010A0005979012352898B4013420ED1143001F03B
:1010B0004FFF024648B1D4F8A4484FF44073617919
:1010C0002068BDE8104000F07FB910BD406BFFF70D
:1010D000DBBF0000704700007FB5124B01250426DE
:1010E000044603600023057400F18402436029462E
:1010F000C0E902330C4B0290143001934FF440735B
:10110000009601F001FF094B04F69442294604F1D0
:101110004C000294CDE900634FF4407301F0C8FF26
:1011200004B070BD383A0008CD100008F10F000877
:101130000A68202383F311880B790B3342F82300CC
:101140004B79133342F823008B7913B10B3342F8F8
:10115000230000F58053C3F8A4180223037400236E
:1011600083F311887047000038B5037F044613B13C
:1011700090F85430ABB90125201D0221FFF730FF54
:1011800004F114006FF00101257700F0CBFC04F1AD
:101190004C0084F854506FF00101BDE8384000F075
:1011A000C1BC38BD10B5012104460430FFF718FF5B
:1011B0000023237784F8543010BD000038B504466E
:1011C0000025143001F0B8FE04F14C00257701F041
:1011D00087FF201D84F854500121FFF701FF2046AE
:1011E000BDE83840FFF750BF90F8803003F060034F
:1011F000202B06D190F881200023212A03D81F2A12
:1012000006D800207047222AFBD1C0E91D3303E035
:10121000034A426707228267C3670120704700BF05
:101220002C22002037B500F58055D5F8A4381A686F
:10123000117804291AD1017C022917D119790123C7
:1012400012898B40134211D100F14C04204602F068
:1012500007F858B101A9204601F04EFFD5F8A4487F
:101260000246019B2179206800F0C0F803B030BD30
:1012700001F10B03F0B550F8236085B004460D462C
:10128000FEB1202383F3118804EB8507301D08216C
:10129000FFF7A6FEFB6806F14C005B691B681BB1FB
:1012A000019001F037FF019803A901F025FF0246E4
:1012B00048B1039B2946204600F098F8002383F3A9
:1012C000118805B0F0BDFB685A691268002AF5D094
:1012D0001B8A013B1340F1D104F18002EAE70000D0
:1012E000133138B550F82140ECB1202383F3118835
:1012F00004F58053D3F8A4281368527903EB8203D2
:10130000DB689B695D6845B104216018FFF768FEE2
:10131000294604F1140001F025FE2046FFF7B4FE33
:10132000002383F3118838BD7047000001F018B91D
:1013300001234022002110B5044600F8303BFFF79E
:1013400091FD0023C4E9013310BD000010B5202336
:10135000044683F311882422416000210C30FFF7FA
:1013600081FD204601F01EF902232370002383F340
:10137000118810BD70B500EB8103054650690E461B
:101380001446DA6018B110220021FFF76BFDA06946
:1013900018B110220021FFF765FD31462846BDE84F
:1013A000704001F011BA000083682022002103F090
:1013B000011310B5044683601030FFF753FD20463B
:1013C000BDE8104001F08CBAF0B4012500EB8104B7
:1013D00047898D40E4683D43A4694581236000232B
:1013E000A2606360F0BC01F0A9BA0000F0B401256E
:1013F00000EB810407898D40E4683D436469058101
:1014000023600023A2606360F0BC01F01FBB0000FA
:1014100070B5022300250446242203702946C0F833
:1014200088500C3040F8045CFFF71CFD204684F81F
:10143000705001F05DF963681B6823B129462046AE
:10144000BDE87040184770BD037880F88C300523E4
:10145000037043681B6810B504460BB1042198471C
:101460000023A36010BD000090F88C204368027038
:101470001B680BB1052118477047000070B590F844
:101480007030044613B1002380F8703004F18002FC
:10149000204601F049FA63689B68B3B994F880303C
:1014A00013F0600535D00021204601F0F3FC002147
:1014B000204601F0E3FC63681B6813B10621204657
:1014C0009847062384F8703070BD2046984700285E
:1014D000E4D0B4F88630A26F9A4288BFA36794F92B
:1014E0008030A56F002B4FF0200380F20381002D88
:1014F00000F0F280092284F8702083F31188002123
:101500002046D4E91D23FFF771FF002383F31188E0
:10151000DAE794F8812003F07F0343EA022340F2E4
:101520000232934200F0C58021D8B3F5807F48D0C5
:101530000DD8012B3FD0022B00F09380002BB2D1AD
:1015400004F1880262670222A267E367C1E7B3F58C
:10155000817F00F09B80B3F5407FA4D194F8823066
:10156000012BA0D1B4F8883043F0020332E0B3F588
:10157000006F4DD017D8B3F5A06F31D0A3F5C0637D
:10158000012B90D86368204694F882205E6894F816
:101590008310B4F88430B047002884D04368636770
:1015A0000368A3671AE0B3F5106F36D040F6024225
:1015B00093427FF478AF5C4B63670223A3670023F9
:1015C000C3E794F88230012B7FF46DAFB4F8883014
:1015D00023F00203A4F88830C4E91D55E56778E7D5
:1015E000B4F88030B3F5A06F0ED194F88230204665
:1015F00084F88A3001F0DAF863681B6813B10121BE
:1016000020469847032323700023C4E91D339CE739
:1016100004F18B0363670123C3E72378042B10D104
:10162000202383F311882046FFF7BEFE85F311883F
:101630000321636884F88B5021701B680BB120462E
:10164000984794F88230002BDED084F88B30042346
:10165000237063681B68002BD6D002212046984770
:10166000D2E794F8843020461D0603F00F010AD516
:1016700001F04CF9012804D002287FF414AF2B4B61
:101680009AE72B4B98E701F033F9F3E794F88230AF
:10169000002B7FF408AF94F8843013F00F01B3D01F
:1016A0001A06204602D501F00DFCADE701F0FEFB65
:1016B000AAE794F88230002B7FF4F5AE94F88430DA
:1016C00013F00F01A0D01B06204602D501F0E2FB6B
:1016D0009AE701F0D3FB97E7142284F8702083F394
:1016E00011882B462A4629462046FFF76DFE85F3D2
:1016F0001188E9E65DB1152284F8702083F3118822
:1017000000212046D4E91D23FFF75EFEFDE60B22F3
:1017100084F8702083F311882B462A4629462046F8
:10172000FFF764FEE3E700BF683A0008603A00088C
:10173000643A000838B590F870300446002B3ED06B
:10174000063BDAB20F2A34D80F2B32D8DFE803F089
:10175000373131082232313131313131313137379E
:10176000856FB0F886309D4214D2C3681B8AB5FBE2
:10177000F3F203FB12556DB9202383F311882B4636
:101780002A462946FFF732FE85F311880A2384F89A
:1017900070300EE0142384F87030202383F3118816
:1017A000002320461A461946FFF70EFE002383F356
:1017B000118838BDC36F03B198470023E7E70021C4
:1017C000204601F067FB0021204601F057FB6368CB
:1017D0001B6813B10621204698470623D7E700006F
:1017E00010B590F870300446142B29D017D8062B6A
:1017F00005D001D81BB110BD093B022BFBD800213D
:10180000204601F047FB0021204601F037FB6368CA
:101810001B6813B1062120469847062319E0152BB3
:10182000E9D10B2380F87030202383F31188002343
:101830001A461946FFF7DAFD002383F31188DAE729
:10184000C3689B695B68002BD5D1C36F03B1984710
:10185000002384F87030CEE7024B0022C3E9003346
:101860009A607047B4230020002382680374054BFC
:101870001B6899689142FBD25A680360426010600D
:1018800058607047B423002008B5202383F31188E3
:10189000037C032B05D0042B0DD02BB983F31188C7
:1018A00008BD436900221A604FF0FF334361FFF720
:1018B000DBFF0023F2E7D0E9003213605A60F3E760
:1018C000002382680374054B1B6899689142FBD81A
:1018D0005A6803604260106058607047B42300206B
:1018E000054B196908741868026853601A6018611A
:1018F00001230374FEF76ABDB42300204B1C30B5EE
:10190000044687B00A4D10D02B6901A8094A00F09F
:1019100025F92046FFF7E4FF049B13B101A800F06E
:1019200059F92B69586907B030BDFFF7D9FFF8E7BF
:10193000B42300208918000838B50C4D04464161D5
:101940002B6981689A68914203D8BDE83840FFF757
:101950008BBF1846FFF7B4FF01232C6101462374A7
:101960002046BDE83840FEF731BD00BFB42300205B
:10197000044B1A681B6990689B68984294BF0020CA
:1019800001207047B423002010B5084C236820695B
:101990001A6854602260012223611A74FFF790FFD5
:1019A00001462069BDE81040FEF710BDB4230020B9
:1019B00008B5FFF7DDFF18B1BDE80840FFF7E4BF49
:1019C00008BD0000FFF7E0BFFEE7000010B50C4CBB
:1019D000FFF742FF00F0B4F880220A49204600F0E9
:1019E0003BF8012344F8180C037400F097FC002323
:1019F00083F3118862B60448BDE8104000F04CB88B
:101A0000DC2300206C3A00087C3A000800F01CB986
:101A1000EFF3118020B9EFF30583202282F31188C0
:101A20007047000010B530B9EFF30584C4F3080423
:101A300014B180F3118810BDFFF7BAFF84F3118849
:101A4000F9E70000034A516853685B1A9842FBD8D3
:101A5000704700BF001000E08260022202827047DF
:101A60008368A3F17C0243F80C2C026943F83C2CF8
:101A7000426943F8382C074A43F81C2CC268A3F18A
:101A8000180043F8102C022203F8082C002203F857
:101A9000072C7047E503000810B5202383F3118855
:101AA000FFF7DEFF00210446FFF746FF002383F324
:101AB0001188204610BD0000024B1B6958610F20A1
:101AC000FFF70EBFB4230020202383F31188FFF714
:101AD000F3BF000008B50146202383F311880820D6
:101AE000FFF70CFF002383F3118808BD49B1064BB3
:101AF00042681B6918605A60136043600420FFF756
:101B0000FDBE4FF0FF307047B423002003689842B9
:101B100006D01A680260506018465961FFF7A4BEEB
:101B20007047000038B504460D462068844200D155
:101B300038BD036823605C604561FFF795FEF4E7FC
:101B4000054B4FF0FF3103F11402C3E905220022D7
:101B5000C3E90712704700BFB423002070B51C4EC4
:101B600005460C46C0E9032301F0B0FB334653F8A9
:101B7000142F9A420DD130620A2C2CBF00190A3062
:101B80002A60C5E90124C6E90555BDE8704001F0A9
:101B900087BB316A431AE31838BF1C469368A342D7
:101BA00002D9081901F08CFB73699A6894420CD829
:101BB0005A68AC602B606A6015609A685D60121BA1
:101BC0009A604FF0FF33F36170BDA41A1B68ECE715
:101BD000B423002038B51B4C636998420DD081684E
:101BE000D0E9003213605A600022C2609A680A4449
:101BF0009A604FF0FF33E36138BD0368224600214D
:101C000042F8143F93425A60C16003D1BDE83840A6
:101C100001F050BB9A688168256A0A449A6001F015
:101C200055FB6369411B9A688A42E5D9AB181D1AB6
:101C3000206A092D98BF01F10A02BDE8384010441E
:101C400001F03EBBB42300202DE9F041184C0027E1
:101C500004F11406656901F039FB236AAA68C11A08
:101C60008A4215D81344D5F80C802362D5E9003296
:101C700013605A606369EF60B34201D101F01AFB4F
:101C800087F311882869C047202383F31188E1E78F
:101C90006169B14209D013441B1ABDE8F0410A2B17
:101CA0002CBFC0180A3001F00BBBBDE8F08100BFAB
:101CB000B423002000207047FEE7000070470000BA
:101CC0004FF0FF307047000002290CD0032904D0E8
:101CD0000129074818BF00207047032A05D8054886
:101CE00000EBC2007047044870470020704700BFF7
:101CF000583B00083C2200200C3B000870B59AB00D
:101D000005460846144601A900F0C2F801A8FFF7ED
:101D1000A1F8431C0022C6B25B001046C5E900349E
:101D200023700323023404F8013C01ABD1B2023426
:101D30008E4201D81AB070BD13F8011B013204F8AD
:101D4000010C04F8021CF1E708B5202383F3118885
:101D50000348FFF767FA002383F3118808BD00BF2B
:101D60007025002090F8803003F01F02012A07D16F
:101D700090F881200B2A03D10023C0E91D3315E020
:101D800003F06003202B08D1B0F884302BB990F811
:101D90008120212A03D81F2A04D8FFF725BA222A36
:101DA000EBD0FAE7034A426707228267C367012044
:101DB000704700BF3322002007B5052917D8DFE898
:101DC00001F0191603191920202383F31188104AF2
:101DD00001210190FFF7CEFA019802210D4AFFF789
:101DE000C9FA0D48FFF7EAF9002383F3118803B01D
:101DF0005DF804FB202383F311880748FFF7B4F94B
:101E0000F2E7202383F311880348FFF7CBF9EBE7D0
:101E1000AC3A0008D03A00087025002038B50C4DC7
:101E20000C4C2A460C4904F10800FFF767FF05F146
:101E3000CA0204F110000949FFF760FF05F5CA72F4
:101E400004F118000649BDE83840FFF757BF00BF4E
:101E5000483E00203C220020943A0008983A0008AE
:101E6000A33A000870B5044608460D46FEF7F2FF97
:101E7000C6B22046013403780BB9184670BD32460D
:101E80002946FEF7D3FF0028F3D10120F6E7000032
:101E90002DE9F04705460C46FEF7DCFF2B49C6B29C
:101EA0002846FFF7DFFF08B10E36F6B2284928466C
:101EB000FFF7D8FF08B11036F6B2632E0BD8DFF863
:101EC0008C80DFF88C90234FDFF894A02E7846B9F1
:101ED0002670BDE8F08729462046BDE8F04701F0AE
:101EE0008DBD252E2ED1072241462846FEF79EFFA6
:101EF00070B9194B224603F1140153F8040B8B42BD
:101F000042F8040BF9D11B78073515341370DDE75F
:101F1000082249462846FEF789FF98B9A21C0F4BB4
:101F2000197802320909C95D02F8041C13F8011B73
:101F300001F00F015345C95D02F8031CF0D11834BC
:101F40000835C3E7013504F8016BBFE7783B0008AB
:101F5000A33A0008963B0008803B000800E8F11F08
:101F60000CE8F11FBFF34F8F044B1A695107FCD1E6
:101F7000D3F810215207F8D1704700BF002000525B
:101F800008B50D4B1B78ABB9FFF7ECFF0B4BDA68CC
:101F9000D10704D50A4A5A6002F188325A60D3F850
:101FA0000C21D20706D5064AC3F8042102F1883273
:101FB000C3F8042108BD00BFA64000200020005245
:101FC0002301674508B5114B1B78F3B9104B1A690B
:101FD000510703D5DA6842F04002DA60D3F81021E5
:101FE000520705D5D3F80C2142F04002C3F80C216A
:101FF000FFF7B8FF064BDA6842F00102DA60D3F867
:102000000C2142F00102C3F80C2108BDA6400020BB
:10201000002000520F289ABF00F580604004002085
:10202000704700004FF400307047000010207047E8
:102030000F2808B50BD8FFF7EDFF00F50033026855
:10204000013204D104308342F9D1012008BD0020BF
:10205000FCE700000F2870B5054645D8FFF7D8FC0F
:10206000224CFFF77FFF0646FFF78AFF4FF0FF3352
:10207000072D6361C4F8143120D82361FFF772FF84
:102080002B0243F02403E360E36843F08003E36042
:1020900023695A07FCD42846FFF764FF4FF4003148
:1020A000FFF7B8FF00F002F93046FFF78BFFFFF7AC
:1020B000B9FC2846BDE87040FFF7BABFC4F810313C
:1020C000FFF750FFA5F108031B0243F02403C4F8F7
:1020D0000C31D4F80C3143F08003C4F80C31D4F83F
:1020E00010315B07FBD4D6E7002070BD0020005202
:1020F0002DE9F84F40EA020305460C461746D8067C
:1021000002D00020BDE8F88F27F01F07DFF8D4B019
:10211000FFF736FF2744BC4203D10120FFF752FFEF
:10212000F0E720222946204601F058FC10B920355E
:102130002034F0E72B4605F120021E68711CE0D127
:1021400004339A42F9D1FFF763FC05F17843234A3F
:10215000B3F5801F224B28BF9A4603F1040338BF12
:102160009046A2F1080228BF9846A3F108033ABF9F
:102170009146DA469946FFF7F5FEC8F80060A5EBF0
:10218000040CD9F8002004F11C0142F00202C9F845
:102190000020221FDAF8006016F00506FAD152F886
:1021A000043F8A424CF80230F4D1BFF34F8FFFF75F
:1021B000D9FE4FF0FF32C8F80020D9F8002022F0F5
:1021C0000202C9F80020FFF72DFC202221462846F4
:1021D00001F004FC0028AAD030469FE714200052EA
:1021E000102100521020005210B5084C237828B15D
:1021F0001BB9FFF7C5FE0123237010BD002BFCD0D7
:102200002070BDE81040FFF7DDBE00BFA6400020F3
:102210000244074BD2B210B5904200D110BD441C0D
:1022200000B253F8200041F8040BE0B2F4E700BF1D
:10223000504000580E4B30B51C6F240405D41C6F61
:102240001C671C6F44F400441C670A4C024423685A
:10225000D2B243F480732360074B904200D130BD6B
:10226000441C51F8045B00B243F82050E0B2F4E79C
:1022700000440258004802585040005807B5012257
:1022800001A90020FFF7C4FF019803B05DF804FB2B
:1022900013B50446FFF7F2FFA04205D0012201A9C1
:1022A00000200194FFF7C6FF02B010BD0144BFF348
:1022B0004F8F064B884204D3BFF34F8FBFF36F8F0E
:1022C0007047C3F85C022030F4E700BF00ED00E087
:1022D000034B1A681AB9034AD2F8D0241A6070471F
:1022E000A84000200040025808B5FFF7F1FF024B5C
:1022F0001868C0F3806008BDA8400020EFF3098390
:10230000054968334A6B22F001024A6383F3098866
:10231000002383F31188704700EF00E0202080F352
:10232000118862B60D4B0E4AD96821F4E0610904A8
:10233000090C0A430B49DA60D3F8FC2042F08072A2
:10234000C3F8FC20084AC2F8B01F116841F001012F
:1023500011601022DA7783F82200704700ED00E068
:102360000003FA0555CEACC5001000E0202310B5DF
:1023700083F311880E4B5B6813F4006314D0F1EE05
:10238000103AEFF309844FF08073683CE361094B26
:10239000DB6B236684F30988FFF7EAFA10B1064B7A
:1023A000A36110BD054BFBE783F31188F9E700BF7C
:1023B00000ED00E000EF00E0F7030008FA0300087A
:1023C00070B5BFF34F8FBFF36F8F1A4A0021C2F869
:1023D0005012BFF34F8FBFF36F8F536943F4003335
:1023E0005361BFF34F8FBFF36F8FC2F88410BFF3F9
:1023F0004F8FD2F8803043F6E074C3F3C900C3F3C3
:102400004E335B0103EA0406014646EA8175013951
:10241000C2F86052F9D2203B13F1200FF2D1BFF382
:102420004F8F536943F480335361BFF34F8FBFF332
:102430006F8F70BD00ED00E0FEE700000A4B0B4817
:102440000B4A90420BD30B4BC11EDA1C121A22F01E
:1024500003028B4238BF00220021FEF703BD53F870
:10246000041B40F8041BECE7743D00087C4200208C
:102470007C4200207C4200207047000070B5D0E90B
:10248000244300224FF0FF359E6804EB42135101B4
:10249000D3F80009002805DAD3F8000940F080409D
:1024A000C3F80009D3F8000B002805DAD3F8000BB5
:1024B00040F08040C3F8000B013263189642C3F825
:1024C0000859C3F8085BE0D24FF00113C4F81C3878
:1024D00070BD000000EB8103D3F80CC02DE9F04380
:1024E000DCF814204E1CD0F89050D2F800E005EB38
:1024F000063605EB4118506870450AD30122D5F81D
:10250000343802FA01F123EA0101C5F83418BDE8B4
:10251000F083AEEB0003BCF81040A34228BF234673
:10252000D8F81849A4B2B3EB840FF0D89468A4F19A
:10253000040959F8047F3760A4EB09071F44042FEE
:10254000F7D81C44034494605360D4E7890141F0F8
:102550002001016103699B06FCD41220FFF772BAC7
:1025600010B50A4C2046FEF7E3FE094BC4F8903044
:10257000084BC4F89430084C2046FEF7D9FE074BB0
:10258000C4F89030064BC4F8943010BDAC40002025
:1025900000000840CC3B00084841002000000440F7
:1025A000D83B000870B503780546012B5DD1494B37
:1025B000D0F89040984259D1474B0E216520D3F86E
:1025C000D82042F00062C3F8D820D3F8002142F0AE
:1025D0000062C3F80021D3F80021D3F8802042F034
:1025E0000062C3F88020D3F8802022F00062C3F894
:1025F0008020D3F8803000F071FC384BE360384B1A
:10260000C4F800380023D5F89060C4F8003EC02319
:1026100023604FF40413A3633369002BFCDA012316
:102620000C203361FFF70EFA3369DB07FCD412206C
:10263000FFF708FA3369002BFCDA00262846A6606B
:10264000FFF71CFF6B68C4F81068DB68C4F81468F7
:10265000C4F81C68002B3AD1224BA3614FF0FF3322
:102660006361A36843F00103A36070BD1E4B9842F1
:10267000C8D1194B0E214D20D3F8D82042F000725A
:10268000C3F8D820D3F8002142F00072C3F800212B
:10269000D3F80021D3F8802042F00072C3F88020E4
:1026A000D3F8802022F00072C3F88020D3F8802075
:1026B000D3F8D82022F08062C3F8D820D3F80021C4
:1026C00022F08062C3F80021D3F8003193E7074B72
:1026D000C3E700BFAC400020004402584014004053
:1026E00003002002003C30C048410020083C30C0BC
:1026F000F8B5D0F89040054600214FF0006620461E
:10270000FFF724FFD5F8941000234FF001128F68D3
:102710004FF0FF30C4F83438C4F81C2804EB4312DF
:1027200001339F42C2F80069C2F8006BC2F8080981
:10273000C2F8080BF2D20B68D5F89020C5F8983093
:10274000636210231361166916F01006FBD1122084
:10275000FFF778F9D4F8003823F4FE63C4F80038A2
:10276000A36943F4402343F01003A3610923C4F891
:102770001038C4F814380B4BEB604FF0C043C4F86A
:10278000103B094BC4F8003BC4F81069C4F8003989
:10279000D5F8983003F1100243F48013C5F898205F
:1027A000A362F8BDA83B000840800010D0F890203C
:1027B00090F88A10D2F8003823F4FE6343EA01133C
:1027C000C2F80038704700002DE9F84300EB8103A0
:1027D000D0F890500C468046DA680FFA81F948012B
:1027E000166806F00306731E022B05EB41134FF02B
:1027F000000194BFB604384EC3F8101B4FF001011E
:1028000004F1100398BF06F1805601FA03F39169B1
:1028100098BF06F5004600293AD0578A04F15801BE
:10282000374349016F50D5F81C180B430021C5F8F8
:102830001C382B180127C3F81019A7405369611ED3
:102840009BB3138A928B9B08012A88BF5343D8F805
:102850009820981842EA034301F140022146C8F843
:102860009800284605EB82025360FFF76FFE08EBE5
:102870008900C3681B8A43EA845348341E436401B9
:102880002E51D5F81C381F43C5F81C78BDE8F883D5
:1028900005EB4917D7F8001B21F40041C7F8001BCE
:1028A000D5F81C1821EA0303C0E704F13F030B4AE3
:1028B0002846214605EB83035A60FFF747FE05EBE8
:1028C0004910D0F8003923F40043C0F80039D5F896
:1028D0001C3823EA0707D7E7008000100004000235
:1028E000D0F894201268C0F89820FFF7C7BD000008
:1028F0005831D0F8903049015B5813F4004004D0AF
:1029000013F4001F0CBF0220012070474831D0F89B
:10291000903049015B5813F4004004D013F4001FB9
:102920000CBF02200120704700EB8101CB68196ABF
:102930000B6813604B6853607047000000EB810325
:1029400030B5DD68AA691368D36019B9402B84BF1C
:10295000402313606B8A1468D0F890201C4402EB6B
:102960004110013C09B2B4FBF3F46343033323F099
:10297000030343EAC44343F0C043C0F8103B2B6851
:1029800003F00303012B0ED1D2F8083802EB4110FB
:1029900013F4807FD0F8003B14BF43F0805343F022
:1029A0000053C0F8003B02EB4112D2F8003B43F069
:1029B0000443C2F8003B30BD2DE9F041D0F89060EF
:1029C00005460C4606EB4113D3F8087B3A07C3F8DB
:1029D000087B08D5D6F814381B0704D500EB810313
:1029E000DB685B689847FA071FD5D6F81438DB0711
:1029F0001BD505EB8403D968CCB98B69488A5A6822
:102A0000B2FBF0F600FB16228AB91868DA68904229
:102A10000DD2121AC3E90024202383F31188214622
:102A20002846FFF78BFF84F31188BDE8F08101236E
:102A300003FA04F26B8923EA02036B81CB68002B53
:102A4000F3D021462846BDE8F041184700EB81034A
:102A50004A0170B5DD68D0F890306C692668E66090
:102A600056BB1A444FF40020C2F810092A6802F03D
:102A70000302012A0AB20ED1D3F8080803EB42146C
:102A800010F4807FD4F8000914BF40F0805040F06B
:102A90000050C4F8000903EB4212D2F8000940F0DC
:102AA0000440C2F800090122D3F8340802FA01F107
:102AB0000143C3F8341870BD19B9402E84BF4020BB
:102AC000206020681A442E8A8419013CB4FBF6F475
:102AD00040EAC44040F00050C6E700002DE9F04154
:102AE000D0F8906004460D4606EB4113D3F8087900
:102AF000C3F80879FB071CD5D6F81038DA0718D5C3
:102B000000EB8103D3F80CC0DCF81430D3F800E0FC
:102B1000DA6896451BD2A2EB0E024FF000081A604D
:102B2000C3F80480202383F31188FFF78FFF88F315
:102B300011883B0618D50123D6F83428AB40134240
:102B400012D029462046BDE8F041FFF7C3BC01235F
:102B500003FA01F2038923EA02030381DCF8083057
:102B6000002BE6D09847E4E7BDE8F0812DE9F84F67
:102B7000D0F8905004466E69AB691E4016F4805838
:102B80006E6103D0BDE8F84FFEF742BC002E12DAAA
:102B9000D5F8003E9F0705D0D5F8003E23F003038B
:102BA000C5F8003ED5F80438204623F00103C5F8E7
:102BB0000438FEF759FC300505D52046FFF75EFCCA
:102BC0002046FEF741FCB1040CD5D5F8083813F0C7
:102BD000060FEB6823F470530CBF43F4105343F417
:102BE000A053EB60320704D56368DB680BB1204665
:102BF0009847F30200F1BA80B70226D5D4F8909036
:102C000000274FF0010A09EB4712D2F8003B03F40A
:102C10004023B3F5802F11D1D2F8003B002B0DDA01
:102C200062890AFA07F322EA0303638104EB87034C
:102C3000DB68DB6813B13946204698470137D4F882
:102C40009430FFB29B689F42DDD9F00619D5D4F8C5
:102C50009000026AC2F30A1702F00F0302F4F012A6
:102C6000B2F5802F00F0CC80B2F5402F09D104EBF3
:102C70008303002200F58050DB681B6A974240F016
:102C8000B2803003D5F8185835D5E90303D50021B3
:102C90002046FFF791FEAA0303D501212046FFF746
:102CA0008BFE6B0303D502212046FFF785FE2F0321
:102CB00003D503212046FFF77FFEE80203D5042158
:102CC0002046FFF779FEA90203D505212046FFF72C
:102CD00073FE6A0203D506212046FFF76DFE2B0224
:102CE00003D507212046FFF767FEEF0103D5082132
:102CF0002046FFF761FE700340F1A980E90703D584
:102D000000212046FFF7EAFEAA0703D5012120464D
:102D1000FFF7E4FE6B0703D502212046FFF7DEFE36
:102D20002F0703D503212046FFF7D8FEEE0603D573
:102D300004212046FFF7D2FEA80603D50521204630
:102D4000FFF7CCFE690603D506212046FFF7C6FE35
:102D50002A0603D507212046FFF7C0FEEB0576D5EE
:102D600020460821BDE8F84FFFF7B8BED4F8909090
:102D700000274FF0010AD4F894305FFA87FB9B6874
:102D80009B453FF639AF09EB4B13D3F8002902F40A
:102D90004022B2F5802F24D1D3F80029002A20DA6E
:102DA000D3F8002942F09042C3F80029D3F8002953
:102DB000002AFBDB5946D4F89000FFF7C7FB2289B5
:102DC0000AFA0BF322EA0303238104EB8B03DB688B
:102DD0009B6813B159462046984759462046FFF74D
:102DE00079FB0137C7E7910701D1D0F80080072AA6
:102DF00002F101029CBF03F8018B4FEA18283DE75E
:102E000004EB830300F58050DA68D2F818C0DCF8D0
:102E10000820DCE9001CA1EB0C0C00218F4208D13A
:102E2000DB689B699A683A449A605A683A445A60E7
:102E300027E711F0030F01D1D0F800808C4501F194
:102E4000010184BF02F8018B4FEA1828E6E7BDE8CC
:102E5000F88F000008B50348FFF788FEBDE808407A
:102E6000FFF784BAAC40002008B50348FFF77EFEA8
:102E7000BDE80840FFF77ABA48410020D0F890300A
:102E800003EB4111D1F8003B43F40013C1F8003BC0
:102E900070470000D0F8903003EB4111D1F80039B1
:102EA00043F40013C1F8003970470000D0F89030A7
:102EB00003EB4111D1F8003B23F40013C1F8003BB0
:102EC00070470000D0F8903003EB4111D1F8003981
:102ED00023F40013C1F8003970470000090100F124
:102EE0006043012203F56143C9B283F8001300F087
:102EF0001F039A4043099B0003F1604303F56143BC
:102F0000C3F880211A60704730B50433039C017206
:102F1000002104FB0325C160C0E90653049B036341
:102F2000059BC0E90000C0E90422C0E90842C0E9ED
:102F30000A11436330BD00000022416AC260C0E94B
:102F40000411C0E90A226FF00101FEF7EBBD000099
:102F5000D0E90432934201D1C2680AB9181D704702
:102F600000207047036919600021C2680132C26005
:102F7000C269134482699342036124BF436A0361B7
:102F8000FEF7C4BD38B504460D46E3683BB162693F
:102F90000020131D1268A3621344E36207E0237A42
:102FA00033B929462046FEF7A1FD0028EDDA38BDE9
:102FB0006FF00100FBE70000C368C269013BC3601A
:102FC0004369134482699342436124BF436A436166
:102FD00000238362036B03B11847704770B5202349
:102FE000044683F31188866A3EB9FFF7CBFF054696
:102FF00018B186F31188284670BDA36AE26A13F8F7
:10300000015B9342A36202D32046FFF7D5FF002362
:1030100083F31188EFE700002DE9F84F04460E46D0
:10302000174698464FF0200989F311880025AA46D3
:10303000D4F828B0BBF1000F09D141462046FFF774
:10304000A1FF20B18BF311882846BDE8F88FD4E9A1
:103050000A12A7EB050B521A934528BF9346BBF102
:10306000400F1BD9334601F1400251F8040B914245
:1030700043F8040BF9D1A36A403640354033A362CC
:10308000D4E90A239A4202D32046FFF795FF8AF338
:103090001188BD42D8D289F31188C9E730465A4613
:1030A000FDF7BAFEA36A5E445D445B44A362E7E7B2
:1030B00010B5029C0433017204FB0321C460C0E913
:1030C00006130023C0E90A33039B0363049BC0E992
:1030D0000000C0E90422C0E90842436310BD0000BB
:1030E000026A6FF00101C260426AC0E90422002254
:1030F000C0E90A22FEF716BDD0E904239A4201D1A5
:10310000C26822B9184650F8043B0B607047002093
:1031100070470000C3680021C2690133C36043697E
:10312000134482699342436124BF436A4361FEF7BB
:10313000EDBC000038B504460D46E3683BB1236999
:1031400000201A1DA262E2691344E36207E0237AB9
:1031500033B929462046FEF7C9FC0028EDDA38BD10
:103160006FF00100FBE7000003691960C268013AD3
:10317000C260C269134482699342036124BF436AF7
:10318000036100238362036B03B11847704700009B
:1031900070B520230D460446114683F31188866AD4
:1031A0002EB9FFF7C7FF10B186F3118870BDA36A6F
:1031B0001D70A36AE26A01339342A36204D3E169FA
:1031C00020460439FFF7D0FF002080F31188EDE797
:1031D0002DE9F84F04460D46904699464FF0200AD7
:1031E0008AF311880026B346A76A4FB9494620469C
:1031F000FFF7A0FF20B187F311883046BDE8F88FB4
:10320000D4E90A073A1AA8EB0607974228BF1746DF
:10321000402F1BD905F1400355F8042B9D4240F87F
:10322000042BF9D1A36A40364033A362D4E90A23C0
:103230009A4204D3E16920460439FFF795FF8BF3E6
:1032400011884645D9D28AF31188CDE729463A46F6
:10325000FDF7E2FDA36A3D443E443B44A362E5E73B
:10326000D0E904239A4217D1C3689BB1836A8BB11A
:10327000043B9B1A0ED01360C368013BC360C36953
:103280001A4483699A42026124BF436A036100239E
:1032900083620123184670470023FBE700F0DAB889
:1032A000034B002258631A610222DA60704700BFA4
:1032B000000C0040014B0022DA607047000C004017
:1032C000014B5863704700BF000C0040014B586A27
:1032D000704700BF000C00404B6843608B68836000
:1032E000CB68C3600B6943614B6903628B694362BE
:1032F0000B6803607047000008B53C4B40F2FF715B
:103300003B48D3F888200A43C3F88820D3F88820A4
:1033100022F4FF6222F00702C3F88820D3F8882045
:10332000D3F8E0200A43C3F8E020D3F808210A4389
:10333000C3F808212F4AD3F808311146FFF7CCFF14
:1033400000F5806002F11C01FFF7C6FF00F5806008
:1033500002F13801FFF7C0FF00F5806002F154016F
:10336000FFF7BAFF00F5806002F17001FFF7B4FFCC
:1033700000F5806002F18C01FFF7AEFF00F5806080
:1033800002F1A801FFF7A8FF00F5806002F1C40177
:10339000FFF7A2FF00F5806002F1E001FFF79CFF5C
:1033A00000F5806002F1FC01FFF796FF02F58C71D9
:1033B00000F58060FFF790FF00F004F90E4BD3F8A2
:1033C000902242F00102C3F89022D3F8942242F0F6
:1033D0000102C3F894220522C3F898204FF06052EE
:1033E000C3F89C20054AC3F8A02008BD0044025839
:1033F00000000258E43B000800ED00E01F00080355
:1034000008B500F0CDFAFEF7E1FA0F4BD3F8DC2057
:1034100042F04002C3F8DC20D3F8042122F040023D
:10342000C3F80421D3F80431084B1A6842F00802AB
:103430001A601A6842F004021A60FEF749FFBDE8FC
:103440000840FEF7EBBC00BF0044025800180248D9
:1034500070470000114BD3F8E82042F00802C3F88F
:10346000E820D3F8102142F00802C3F810210C4ADA
:10347000D3F81031D36B43F00803D363C722094B51
:103480009A624FF0FF32DA6200229A615A63DA6080
:103490005A6001225A611A60704700BF0044025806
:1034A0000010005C000C0040094A08B51169D3689F
:1034B0000B40D9B29B076FEA0101116107D52023A8
:1034C00083F31188FEF7A2FA002383F3118808BD65
:1034D000000C00403A4B4FF0FF31D3F8802062F0EF
:1034E0000042C3F88020D3F8802002F00042C3F8E5
:1034F0008020D3F88020D3F88420C3F88410D3F838
:1035000084200022C3F88420D3F88400D86F40F0D0
:10351000FF4040F4FF0040F43F5040F03F00D867C8
:10352000D86F20F0FF4020F4FF0020F43F5020F03F
:103530003F00D867D86FD3F888006FEA40506FEA31
:103540005050C3F88800D3F88800C0F30A00C3F8CD
:103550008800D3F88800D3F89000C3F89010D3F80F
:103560009000C3F89020D3F89000D3F89400C3F8EB
:103570009410D3F89400C3F89420D3F89400D3F8AF
:103580009800C3F89810D3F89800C3F89820D3F89F
:103590009800D3F88C00C3F88C10D3F88C00C3F8D3
:1035A0008C20D3F88C00D3F89C00C3F89C10D3F87F
:1035B0009C10C3F89C20D3F89C3000F0C9B900BF20
:1035C00000440258614B0122C3F80821604BD3F834
:1035D000F42042F00202C3F8F420D3F81C2142F098
:1035E0000202C3F81C210222D3F81C31594BDA60C5
:1035F0005A689104FCD5584A1A6001229A60574AC9
:10360000DA6000221A614FF440429A61514B9A6984
:103610009204FCD51A6842F480721A604C4B1A6FFF
:1036200012F4407F04D04FF480321A6700221A67E8
:103630001A6842F001021A60454B1A685007FCD51F
:1036400000221A611A6912F03802FBD101211960B7
:103650004FF0804159605A67414ADA62414A1A6123
:103660001A6842F480321A60394B1A689103FCD50B
:103670001A6842F480521A601A689204FCD53A4AD9
:103680003A499A6200225A6319633949DA639963A5
:103690005A64384A1A64384ADA621A6842F0A85200
:1036A0001A602B4B1A6802F02852B2F1285FF9D148
:1036B00048229A614FF48862DA6140221A622F4AE6
:1036C000DA644FF080521A652D4A5A652D4A9A6580
:1036D00032232D4A1360136803F00F03022BFAD133
:1036E0001B4B1A6942F003021A611A6902F0380290
:1036F000182AFAD1D3F8DC2042F00052C3F8DC20BB
:10370000D3F8042142F00052C3F80421D3F8042175
:10371000D3F8DC2042F08042C3F8DC20D3F8042147
:1037200042F08042C3F80421D3F80421D3F8DC200E
:1037300042F00042C3F8DC20D3F8042142F00042FA
:10374000C3F80421D3F80431704700BF0080005152
:10375000004402580048025800C000F00200000176
:103760000000FF0100889008322060006302090118
:103770001D02040047040508FD0BFF012000002086
:103780000010E00000010100002000524FF0B042A4
:1037900008B5D2F8883003F00103C2F8883023B1AD
:1037A000044A13680BB150689847BDE80840FEF71B
:1037B000DDBD00BFFC4100204FF0B04208B5D2F89B
:1037C000883003F00203C2F8883023B1044A9368BA
:1037D0000BB1D0689847BDE80840FEF7C7BD00BFF1
:1037E000FC4100204FF0B04208B5D2F8883003F019
:1037F0000403C2F8883023B1044A13690BB150693D
:103800009847BDE80840FEF7B1BD00BFFC4100206D
:103810004FF0B04208B5D2F8883003F00803C2F880
:10382000883023B1044A93690BB1D0699847BDE849
:103830000840FEF79BBD00BFFC4100204FF0B042A6
:1038400008B5D2F8883003F01003C2F8883023B1ED
:10385000044A136A0BB1506A9847BDE80840FEF766
:1038600085BD00BFFC4100204FF0B04310B5D3F838
:10387000884004F47872C3F88820A30604D5124A5D
:10388000936A0BB1D06A9847600604D50E4A136B51
:103890000BB1506B9847210604D50B4A936B0BB1C3
:1038A000D06B9847E20504D5074A136C0BB1506CF6
:1038B0009847A30504D5044A936C0BB1D06C984784
:1038C000BDE81040FEF752BDFC4100204FF0B04370
:1038D00010B5D3F8884004F47C42C3F88820620510
:1038E00004D5164A136D0BB1506D9847230504D5C6
:1038F000124A936D0BB1D06D9847E00404D50F4A7E
:10390000136E0BB1506E9847A10404D50B4A936E09
:103910000BB1D06E9847620404D5084A136F0BB1FF
:10392000506F9847230404D5044A936F0BB1D06FAE
:103930009847BDE81040FEF719BD00BFFC410020CC
:1039400008B5FFF7B1FDBDE80840FEF70FBD000068
:10395000062108B50846FFF7C1FA06210720FFF740
:10396000BDFA06210820FFF7B9FA06210920FFF762
:10397000B5FA06210A20FFF7B1FA06211720FFF752
:10398000ADFA06212820FFF7A9FA09217A20FFF7CE
:10399000A5FA07213220BDE80840FFF79FBA0000D2
:1039A00008B5FFF797FD00F00BF8FDF7BFFCFDF73A
:1039B00091FBFFF74DFDBDE80840FFF76FBC00002D
:1039C0000023054A19460133102BC2E9001102F108
:1039D0000802F8D1704700BFFC41002010B5013942
:1039E0000244904201D1002005E0037811F8014F14
:1039F000A34201D0181B10BD0130F2E7034611F8B5
:103A0000012B03F8012B002AF9D1704753544D3391
:103A10003248373F3F3F0053544D333248373433F9
:103A20002F3735330000000001105A0003105900F1
:103A3000012058000320560000000000511000082B
:103A40003D1000087910000865100008711000088A
:103A50005D100008491000083510000885100008A6
:103A60000000000001000000000000006D61696EB0
:103A70000000000069646C6500000000743A0008F2
:103A8000F82300207025002001000000C91900085B
:103A9000000000006D526F0025424F415244252D19
:103AA000424C002553455249414C2500020000007C
:103AB0000000000071120008E11200084000400000
:103AC000183E0020283E00200200000000000000F8
:103AD000030000000000000029130008000000009F
:103AE00010000000383E002000000000010000002F
:103AF00000000000AC40002001010200B91D0008D8
:103B0000C91C0008651D0008491D0008430000008D
:103B1000143B000809024300020100C032090400FE
:103B2000000102020100052400100105240100012A
:103B3000042402020524060001070582030800FF91
:103B400009040100020A000000070501024000000C
:103B5000070581024000000012000000603B0008E1
:103B60001201100102000040091241570002010237
:103B7000030100000403090425424F41524425007B
:103B80006D526F436F6E74726F6C5A65726F436CD7
:103B90006173736963003031323334353637383905
:103BA0004142434445460000000000007D140008E7
:103BB00035170008E117000840004000E4410020EC
:103BC000E441002001000000F441002080000000DA
:103BD0004001000008000000000100000004000097
:103BE000080000000000802A00000000AAAAAAAA7B
:103BF00000000024FFFF00000000000000A00A00F9
:103C00004401000000000000AAAAAAAA00000000C7
:103C1000FFFF0000000000000000000000000000A6
:103C200000000000AAAAAAAA00000000FFFF0000EE
:103C30000000000000000000004010000000000034
:103C4000AAAA8AAA00401000FFFF0000000000009E
:103C5000000000000000004000000000AAAAAAAA7C
:103C600000000040FFFF0000000000000000000016
:103C70000100100000000000AAAAAAAA010010007A
:103C8000FFFF0000000000000000000040000400F2
:103C900000000000AAAAAAAA40000400FFFF00003A
:103CA0000000000000000000000000000000000014
:103CB000AAAAAAAA00000000FFFF0000000000005E
:103CC000000000000000000000000000AAAAAAAA4C
:103CD00000000000FFFF00000000000000000000E6
:103CE0000000000000000000AAAAAAAA000000002C
:103CF000FFFF0000000000000000000000000000C6
:103D000000000000AAAAAAAA00000000FFFF00000D
:103D10000000000000000000FE03000000000000A2
:103D200000001E0000000000FF0000000000000076
:103D30000C3A00083F00000050040000173A000849
:103D40003F00000000960000000008009600000000
:103D50000008000004000000743B000800000000A0
:103D60000000000000000000000000000000000053
:043D7000000000004F
:00000001FF
